BL51 BANKED LINKER/LOCATER V6.00                                                        01/16/2018  10:33:28  PAGE 1


BL51 BANKED LINKER/LOCATER V6.00, INVOKED BY:
C:\KEIL\C51\BIN\BL51.EXE main.obj TO MA82G5Dxx RAMSIZE (256)


MEMORY MODEL: SMALL


INPUT MODULES INCLUDED:
  main.obj (MAIN)
  C:\KEIL\C51\LIB\C51S.LIB (?C_STARTUP)


LINK MAP OF MODULE:  MA82G5Dxx (MAIN)


            TYPE    BASE      LENGTH    RELOCATION   SEGMENT NAME
            -----------------------------------------------------

            * * * * * * *   D A T A   M E M O R Y   * * * * * * *
            REG     0000H     0008H     ABSOLUTE     "REG BANK 0"
            DATA    0008H     0013H     UNIT         ?DT?MAIN
            IDATA   001BH     0001H     UNIT         ?STACK

            * * * * * * *   C O D E   M E M O R Y   * * * * * * *
            CODE    0000H     0003H     ABSOLUTE     
            CODE    0003H     001DH     UNIT         ?PR?INT_UART0?MAIN
                    0020H     0003H                  *** GAP ***
            CODE    0023H     0003H     ABSOLUTE     
            CODE    0026H     0036H     UNIT         ?PR?UART0_SHOW_UID?MAIN
            CODE    005CH     001BH     UNIT         ?PR?INITIAL_UART0?MAIN
            CODE    0077H     000FH     UNIT         ?PR?MAIN?MAIN
            CODE    0086H     000DH     UNIT         ?PR?_UART0_SEND_BYTE?MAIN
            CODE    0093H     000CH     UNIT         ?C_C51STARTUP



OVERLAY MAP OF MODULE:   MA82G5Dxx (MAIN)


SEGMENT
  +--> CALLED SEGMENT
---------------------
?C_C51STARTUP
  +--> ?PR?MAIN?MAIN

?PR?MAIN?MAIN
  +--> ?PR?INITIAL_UART0?MAIN
  +--> ?PR?UART0_SHOW_UID?MAIN

?PR?UART0_SHOW_UID?MAIN
  +--> ?PR?_UART0_SEND_BYTE?MAIN



SYMBOL TABLE OF MODULE:  MA82G5Dxx (MAIN)

  VALUE           TYPE          NAME
  ----------------------------------
BL51 BANKED LINKER/LOCATER V6.00                                                      01/16/2018  10:33:28  PAGE 2



  -------         MODULE        MAIN
  C:0000H         SYMBOL        _ICE_DUMMY_
  D:0008H         PUBLIC        flag_Tx0_Busy
  D:0096H         PUBLIC        BOREV
  D:0090H         PUBLIC        P1
  D:00A0H         PUBLIC        P2
  D:00E7H         PUBLIC        ISPCR
  D:00C0H         PUBLIC        XICON
  D:00B0H         PUBLIC        P3
  D:00E8H         PUBLIC        P4
  D:00F8H         PUBLIC        P6
  D:00ACH         PUBLIC        SFRPI
  B:00A8H.7       PUBLIC        EA
  D:00A8H         PUBLIC        IE
  D:00B8H         PUBLIC        IP0L
  C:005CH         PUBLIC        Initial_UART0
  D:00C7H         PUBLIC        CKCON0
  D:00CBH         PUBLIC        RCAP2H
  D:00D8H         PUBLIC        CCON
  D:00CAH         PUBLIC        RCAP2L
  C:0077H         PUBLIC        main
  D:00E6H         PUBLIC        SCMD
  D:00E3H         PUBLIC        IFADRH
  C:0086H         PUBLIC        _UART0_Send_Byte
  D:00E5H         PUBLIC        IFMT
  D:00E4H         PUBLIC        IFADRL
  C:0026H         PUBLIC        UART0_Show_UID
  D:0088H         PUBLIC        TCON
  C:0003H         PUBLIC        INT_UART0
  D:0009H         PUBLIC        UID_Code
  B:00A8H.4       PUBLIC        ES0
  B:0098H.0       PUBLIC        RI0
  B:0098H.1       PUBLIC        TI0
  D:00CDH         PUBLIC        TH2
  D:0019H         PUBLIC        tmp
  D:00CCH         PUBLIC        TL2
  D:00E2H         PUBLIC        IFD
  B:00C8H.2       PUBLIC        TR2
  D:0099H         PUBLIC        S0BUF
  D:0087H         PUBLIC        PCON0
  D:0098H         PUBLIC        S0CON
  D:00C9H         PUBLIC        T2MOD
  D:00C8H         PUBLIC        T2CON
  D:001AH         PUBLIC        i
  D:00D0H         PUBLIC        PSW
  -------         PROC          INT_UART0
  C:0003H         LINE#         30
  C:0007H         LINE#         32
  C:000AH         LINE#         33
  C:000CH         LINE#         35
  C:0011H         LINE#         36
  C:0011H         LINE#         37
  C:0013H         LINE#         38
  C:0018H         LINE#         39
  C:001BH         LINE#         40
  C:001BH         LINE#         41
BL51 BANKED LINKER/LOCATER V6.00                                                      01/16/2018  10:33:28  PAGE 3


  -------         ENDPROC       INT_UART0
  -------         PROC          INITIAL_UART0
  C:005CH         LINE#         44
  C:005CH         LINE#         45
  C:005CH         LINE#         46
  C:005FH         LINE#         47
  C:0062H         LINE#         48
  C:0065H         LINE#         49
  C:0068H         LINE#         50
  C:006BH         LINE#         51
  C:006EH         LINE#         52
  C:0071H         LINE#         53
  C:0073H         LINE#         54
  C:0076H         LINE#         55
  -------         ENDPROC       INITIAL_UART0
  -------         PROC          _UART0_SEND_BYTE
  D:0007H         SYMBOL        dta
  C:0086H         LINE#         57
  C:0086H         LINE#         58
  C:0086H         LINE#         59
  C:0089H         LINE#         60
  C:008BH         LINE#         61
  C:008EH         LINE#         62
  C:0092H         LINE#         63
  -------         ENDPROC       _UART0_SEND_BYTE
  -------         PROC          UART0_SHOW_UID
  C:0026H         LINE#         65
  C:0026H         LINE#         66
  C:0026H         LINE#         67
  C:0029H         LINE#         68
  C:002CH         LINE#         69
  C:002FH         LINE#         70
  C:0032H         LINE#         71
  C:0035H         LINE#         73
  C:0037H         LINE#         74
  C:0037H         LINE#         75
  C:003AH         LINE#         76
  C:003DH         LINE#         77
  C:0044H         LINE#         78
  C:0049H         LINE#         79
  C:004BH         LINE#         80
  C:0054H         LINE#         81
  C:0057H         LINE#         82
  C:0059H         LINE#         83
  C:005BH         LINE#         84
  -------         ENDPROC       UART0_SHOW_UID
  -------         PROC          MAIN
  C:0077H         LINE#         87
  C:0077H         LINE#         88
  C:0077H         LINE#         89
  C:007AH         LINE#         90
  C:007DH         LINE#         91
  C:007FH         LINE#         92
  C:0081H         LINE#         95
  C:0084H         LINE#         98
  -------         ENDPROC       MAIN
  -------         ENDMOD        MAIN
BL51 BANKED LINKER/LOCATER V6.00                                                      01/16/2018  10:33:28  PAGE 4



Program Size: data=28.0 xdata=0 code=156
LINK/LOCATE RUN COMPLETE.  0 WARNING(S),  0 ERROR(S)
